S0190000526F6569626F6F74204669726D776172652E737265636B
S11300001DC037C036C096C134C0B9C08CC0A1C0B1
S113001030C02FC02EC016C22CC02BC02AC029C08D
S113002028C03FC226C025C024C023C022C021C08E
S113003020C01FC01EC01DC01CC01BC011241FBE79
S1130040CFEFD2E0DEBFCDBF11E0A0E0B1E0E4E449
S1130050F7E102C005900D92A633B107D9F721E06C
S1130060A6E3B1E001C01D92A135B207E1F739D88A
S113007067CBC6CF1092920083E380939100E6E9A8
S1130080F0E080818D7F808388E18093950086E015
S113009080939400089540E0342FB29913C0B2992C
S11300A030C0832FE7EEF3E03197F1F700C0000092
S11300B08F5FB29903C08832A9F727C0B29902C0F2
S11300C08732C8F4B29BE9CFB29B1DC0942FE7EEF0
S11300D0F3E03197F1F700C000009F5F26B3822F51
S11300E0847022FF03C0983291F712C0B29BD5CF1F
S11300F0973298F2089581E0089581E0089580E0B0
S1130100089586B3DFCF86B3C8CFB29BF6CFDACFDC
S1130110B299F5CFC2CFBFDF8823E9F30895BBDFDF
S11301208111FDCF08951F920F920FB60F921124E3
S11301308F9380914C01882319F0813019F003C00A
S1130140D99801C0DB988F910F900FBE0F901F902C
S113015018951F920F920FB60F9211248F938091CE
S11301604C01882319F0813019F003C0DA9801C0DA
S1130170DF988F910F900FBE0F901F9018951F92CC
S11301800F920FB60F9211242F933F938F939F9347
S113019080914C01882319F08130C9F02EC081E090
S11301A080934C01809133018111DB9A809132015B
S11301B08111DF9A80912C0190912D019BBD8ABD04
S11301C080912A0190912B0199BD88BD16C010928F
S11301D04C01809135018111D99A809134018111AA
S11301E0DA9A80913001909131019BBD8ABD809152
S11301F02E0190912F0199BD88BD2091300130913D
S1130200310180912801909129012817390769F457
S113021080914A018E3F30F480914A018F5F809330
S11302204A0108C01092350105C010924A0181E0CC
S11302308093350120912E0130912F018091260168
S1130240909127012817390769F4809149018E3F5D
S113025030F4809149018F5F8093490108C0109266
S1130260340105C01092490181E08093340120914A
S11302702C0130912D0180912401909125012817A2
S1130280390769F4809148018E3F30F48091480128
S11302908F5F8093480108C01092330105C010920B
S11302A0480181E08093330120912A0130912B0190
S11302B080912201909123012817390769F48091D4
S11302C047018E3F30F4809147018F5F809347014F
S11302D008C01092320105C01092470181E080935A
S11302E032018091300190913101909329018093E2
S11302F0280180912E0190912F01909327018093E2
S1130300260180912C0190912D01909325018093D9
S1130310240180912A0190912B01909323018093D1
S113032022019F918F913F912F910F900FBE0F90BB
S11303301F9018951F920F920FB60F9211242F93AE
S11303404F935F938F939F9380914B01811111C0C1
S1130350B19B0FC018BE12BE10923E0110923D0117
S11303601092400110923F0181E080934B01109262
S1130370460180914B01813011F5B19920C018BE1E
S113038022B780913F0190914001409143015091E7
S11303904401840F951F820F911D96958795909324
S11303A044018093430182E080934B0181E0809378
S11303B0450180B58D7F80BD80B5816080BD809111
S11303C04B01823079F4B09B0DC018BE12BE10925E
S11303D03E0110923D011092400110923F0183E0D2
S11303E080934B0180914B01833009F5B0991FC074
S11303F018BE22B780913D0190913E014091410188
S113040050914201840F951F820F911D96958795F7
S1130410909342018093410110924B0181E08093BB
S1130420450180B58E7F80BD80B5826080BD1ABED7
S11304309F918F915F914F912F910F900FBE0F90CD
S11304401F9018951F920F920FB60F9211248F933D
S11304509F9318BE80913D0190913E0181509F4F22
S113046090933E0180933D0180913F019091400122
S113047081509F4F9093400180933F0180914601AA
S11304808F3F31F0809146018F5F8093460102C017
S1130490109245019F918F910F900FBE0F901F9066
S11304A018951F920F920FB60F9211248F939F935A
S11304B09BB381E089278BBB9F918F910F900FBED7
S11304C00F901F9018954F925F926F927F92AF9208
S11304D0BF92CF92DF92EF92FF920F931F93CF932D
S11304E0DF93CDB7DEB729013A012E153F0540074A
S11304F051073CF0B22FA52DF62DE72DA801970149
S113050004C0BE2DAF2DF02FE12F621773078407AF
S113051095075CF02B2F3A2F4F2F5E2F621773072E
S11305208407950714F49B01AC01CA01B90164194D
S113053075098609970929893A894B895C892A1999
S11305403B094C095D092AD8B22FA32FF42FE52FBC
S1130550A801970124193509460957096B2F7A2FE9
S11305608F2F9E2FFFD7CA01B9016A0D7B1D8C1DE9
S11305709D1DDF91CF911F910F91FF90EF90DF9020
S1130580CF90BF90AF907F906F905F904F90089501
S11305904F925F926F927F92AF92BF92CF92DF920F
S11305A0EF92FF920F931F9320910C0130910D0154
S11305B0A0900E01B0900F01C12CD12C29011F92E3
S11305C01F925F922F93E12CF12C8701EA9420E093
S11305D030E0A90178DF0F900F900F900F90709387
S11305E03101609330011F910F91FF90EF90DF90E4
S11305F0CF90BF90AF907F906F905F904F90089591
S11306004F925F926F927F92AF92BF92CF92DF929E
S1130610EF92FF920F931F932091080130910901EB
S1130620A0900A01B0900B01C12CD12C29011F927A
S11306301F925F922F93E12CF12C8701EA9420E022
S113064030E0A90140DF0F900F900F900F9070934E
S11306502F0160932E011F910F91FF90EF90DF9077
S1130660CF90BF90AF907F906F905F904F90089520
S11306704F925F926F927F92AF92BF92CF92DF922E
S1130680EF92FF920F931F93209104013091050183
S1130690A0900601B0900701C12CD12C29011F9212
S11306A01F925F922F93E12CF12C8701EA9420E0B2
S11306B030E0A90108DF0F900F900F900F90709316
S11306C02D0160932C011F910F91FF90EF90DF900B
S11306D0CF90BF90AF907F906F905F904F900895B0
S11306E04F925F926F927F92AF92BF92CF92DF92BE
S11306F0EF92FF920F931F9320910001309101011B
S1130700A0900201B0900301C12CD12C29011F92A9
S11307101F925F922F93E12CF12C8701EA9420E041
S113072030E0A901D0DE0F900F900F900F907093DE
S11307302B0160932A011F910F91FF90EF90DF909E
S1130740CF90BF90AF907F906F905F904F9008953F
S1130750AF92BF92CF92DF92EF92FF920F931F93CB
S1130760E0901801F090190120911A0130911B01B9
S1130770609143017091440100E010E040E050E0DA
S113078080E090E01F921F921F92EFE7EF930F2EED
S1130790F1E8AF2EBB24BA94CB2CDB2CF02D93DEE6
S11307A00F900F900F900F90862F9EE0960F9D3123
S11307B0E0F02091160130911701409143015091CE
S11307C04401245631092417350780F42091160179
S11307D03091170140914301509144012C593F4FEE
S11307E04217530718F480E001C080E01F910F9175
S11307F0FF90EF90DF90CF90BF90AF900895AF92AD
S1130800BF92CF92DF92EF92FF920F931F93E090EB
S11308101201F0901301209114013091150160919F
S113082041017091420100E010E040E050E080E0BE
S113083090E01F921F921F92EFE7EF930F2EF1E8C3
S1130840AF2EBB24BA94CB2CDB2CF02D3CDE0F90C6
S11308500F900F900F90862F9EE0960F9D31E0F041
S113086020911001309111014091410150914201B8
S1130870245631092417350780F420911001309152
S1130880110140914101509142012C593F4F4217AF
S1130890530718F480E001C080E01F910F91FF908E
S11308A0EF90DF90CF90BF90AF900895AF92BF923A
S11308B0CF92DF92EF92FF920F931F93811102C0A8
S11308C0662319F016160CF041C020911C0180918A
S11308D03C018F3FE9F480912101422F50E090E0E8
S11308E0BA0161587F4F6817790724F48091210178
S11308F0821B12C06091210170E08FE790E0841B9D
S1130900950B681779073CF480912101820F04C08C
S11309108091210101C08FE78093210180913C01E6
S11309208F3F71F030913C01822F90E0830F911D35
S11309308F3F910509F034F480913C01820F03C08C
S11309408FEF01C08FEF80933C0111C166231CF42B
S1130950811101C08CE940911C01A0901C01BB24B1
S1130960A1940CF4B0940B2C000CCC08DD08682F77
S1130970880F770B880B990B042F042E000C110B96
S1130980220B330B3F932F931F934F931FE7E12EBB
S1130990F12C00E010E021E83FEF4FEF5FEF93DD33
S11309A00F900F900F900F90462F440F80913C01B1
S11309B090913C012091210130912101803F30F43C
S11309C0903120F0203F10F4303100F580913C014B
S11309D091E0803F08F490E090933B0180913C01CA
S11309E091E0803108F090E090933A0180912101E8
S11309F091E0803F08F490E090931E0180912101E2
S1130A0091E0803108F090E09093390180913C01AD
S1130A108031C8F480912101E62F062E000CFF0BD3
S1130A2090E08E1B9F0B181619065CF5209121018E
S1130A3030E02E1B3F0B2F3F31052CF59091210107
S1130A40961B692F25C080913C01803FB8F020910E
S1130A502101862F062E000C990BFC01E20FF11DDB
S1130A60EF3FF10594F420912101820F911D181696
S1130A7019066CF490912101690F0AC0609121015B
S1130A8007C060E005C06FEF03C06FEF01C060E016
S1130A906093210180912101803FC0F080913C014D
S1130AA0642F042E000C770B90E0861B970B18160E
S1130AB0190654F520913C0130E0261B370B2F3FDB
S1130AC0310524F580913C01841B25C080912101CE
S1130AD08031B8F420913C01842F042E000C990B32
S1130AE0BC01620F711D1616170694F420913C0187
S1130AF0820F911D8F3F91056CF480913C01840F0E
S1130B000AC080913C0107C080E005C08FEF03C09C
S1130B1080E001C08FEF80933C0180913C01909173
S1130B203C012091210130912101803F00F5903159
S1130B30F0F0203FE0F43031D0F080913B0181307F
S1130B4019F48FEF8093210180913A01813011F4DF
S1130B501092210180911E01813019F48FEF80934E
S1130B603C0180913901813011F410923C011F91B4
S1130B700F91FF90EF90DF90CF90BF90AF900895CA
S1130B80AF92BF92CF92DF92EF92FF920F931F9397
S1130B90811102C0662319F066230CF041C0209134
S1130BA01C0180911F018F3FE9F480912001422FA5
S1130BB050E090E0BA0161587F4F6817790724F438
S1130BC080912001821B12C06091200170E08FE7A8
S1130BD090E0841B950B681779073CF48091200101
S1130BE0820F04C08091200101C08FE7809320010F
S1130BF080911F018F3F71F030911F01822F90E08F
S1130C00830F911D8F3F910509F034F480911F01EA
S1130C10820F03C08FEF01C08FEF80931F0111C1BA
S1130C2016161CF4811101C08CE940911C01A0909E
S1130C301C01BB24A1940CF4B0940B2C000CCC0824
S1130C40DD08682F880F770B880B990B042F042E6F
S1130C50000C110B220B330B3F932F931F934F93D5
S1130C601FE7E12EF12C00E010E021E83FEF4FEF09
S1130C705FEF29DC0F900F900F900F90462F440FD9
S1130C8080911F0190911F0120912001309120013A
S1130C90803F30F4903120F0203F10F4303100F5E3
S1130CA080911F0191E0803F08F490E09093380117
S1130CB080911F0191E0803108F090E0909337011A
S1130CC08091200191E0803F08F490E090931D0111
S1130CD08091200191E0803108F090E090933601FA
S1130CE080911F018031C8F480912001E62F062EE7
S1130CF0000CFF0B90E08E1B9F0B181619065CF579
S1130D002091200130E02E1B3F0B2F3F31052CF5A5
S1130D1090912001961B692F25C080911F01803F6F
S1130D20B8F020912001862F062E000C990BFC01AF
S1130D30E20FF11DEF3FF10594F420912001820FA1
S1130D40911D181619066CF490912001690F0AC0C0
S1130D506091200107C060E005C06FEF03C06FEF32
S1130D6001C060E06093200180912001803FC0F0C9
S1130D7080911F01642F042E000C770B90E0861BDA
S1130D80970B1816190654F520911F0130E0261B05
S1130D90370B2F3F310524F580911F01841B25C09B
S1130DA0809120018031B8F420911F01842F042EFA
S1130DB0000C990BBC01620F711D1616170694F4F2
S1130DC020911F01820F911D8F3F91056CF480913A
S1130DD01F01840F0AC080911F0107C080E005C075
S1130DE08FEF03C080E001C08FEF80931F018091DB
S1130DF01F0190911F012091200130912001803F1B
S1130E0000F59031F0F0203FE0F43031D0F08091E3
S1130E103801813019F48FEF8093200180913701DC
S1130E20813011F41092200180911D01813019F458
S1130E308FEF80931F0180913601813011F410925D
S1130E401F011F910F91FF90EF90DF90CF90BF9003
S1130E50AF900895823068F4E9ECF0E09081927FDD
S1130E6090831092C5001092C4006BB3682B6BBBC7
S1130E700895682F70E088E09DE360D38091C400FA
S1130E809091C5008617970769F0E9ECF0E080813E
S1130E908D6080831092C7001092C6007093C500C5
S1130EA06093C40008950F931F93CF93DF93EC01D5
S1130EB08B011CC04DDC833364F028813981265FAB
S1130EC03F4F39832883EFE1FEE43197F1F700C007
S1130ED000008E3C5CF4888199810A979983888309
S1130EE08FE19EE40197F1F700C00000D4D8882375
S1130EF009F388819981F8019183808388E0AADFCE
S1130F000ED9FFEF29E688E1F15020408040E1F757
S1130F1000C0000081E09EDFDF91CF911F910F910F
S1130F20089588E097DFFBD82FEF89E698E12150F8
S1130F3080409040E1F700C0000081E08BDFEBD8F7
S1130F4088E088DF809143019091440190931701D8
S1130F5080931601E4D82FEF89E698E12150804070
S1130F609040E1F700C0000081E074DFD4D888E04D
S1130F7071DF809143019091440190931B01809310
S1130F801A01CDD82FEF89E698E121508040904096
S1130F90E1F700C0000081E05DDFBDD888E05ADFE2
S1130FA08091430190914401909319018093180119
S1130FB0B6D82FEF89E698E1215080409040E1F7C0
S1130FC000C0000081E046DFA6D888E043DF8091BE
S1130FD041019091420190931101809310019FD897
S1130FE02FEF89E698E1215080409040E1F700C05E
S1130FF0000081E02FDF8FD888E02CDF8091410151
S113100090914201909315018093140188D82FEF99
S113101089E698E1215080409040E1F700C000004B
S113102081E018DF78D888E015DF80914101909144
S11310304201909313018093120171D82FEF89E636
S113104098E1215080409040E1F700C0000081E029
S113105001DF6CE071E080E391E025DF6EE071E098
S113106080E391E020DF6AE071E08EE291E01BDF33
S113107068E071E08EE291E016DF64E071E08CE2FA
S113108091E011DF66E071E08CE291E00CDF62E058
S113109071E08AE291E007DF60E071E08AE291E0CA
S11310A002DF81E0D7DE37D888E0D4DE51DB8E3C26
S11310B024F482E080931C0109C0833324F084E08B
S11310C080931C0103C083E080931C0128D82FEF78
S11310D089E698E1215080409040E1F700C000008B
S11310E00895CF93DF9300D0CDB7DEB788ED80931A
S11310F071001092730088E090E0FCD2893893412B
S113110008F467C060911A0170911B0180E090E0BF
S113111004D3609118017091190182E090E0FDD22E
S1131120609116017091170188E190E0F6D2609108
S113113014017091150184E090E0EFD260911201E6
S11311407091130186E090E0E8D2609110017091F3
S113115011018AE190E0E1D260910E0170910F01DA
S113116088E090E0DAD260910C0170910D018AE080
S113117090E0D3D260910A0170910B018CE090E071
S1131180CCD260910801709109018EE090E0C5D243
S1131190609106017091070180E190E0BED26091F8
S11311A004017091050182E190E0B7D260910201DF
S11311B07091030184E190E0B0D2609100017091DC
S11311C0010186E190E0A9D260911C018CE190E0DC
S11311D096D280E090E08ED290931B0180931A0106
S11311E082E090E087D2909319018093180188E1FE
S11311F090E080D2909317018093160184E090E0F0
S113120079D2909315018093140186E090E072D214
S113121090931301809312018AE190E06BD2909332
S113122011018093100188E090E064D290930F0143
S113123080930E018AE090E05DD290930D0180933B
S11312400C018CE090E056D290930B0180930A013C
S11312508EE090E04FD2909309018093080180E1E1
S113126090E048D2909307018093060182E190E0D8
S113127041D2909305018093040184E190E03AD235
S1131280909303018093020186E190E033D290931E
S11312900101809300018CE190E024D280931C0131
S11312A08EB588618EBD80E197E295BD84BD8EB513
S11312B082608EBD8FB186628FB98CED95E09BBD47
S11312C08ABD80E496E099BD88BD83B7826083BF00
S11312D089B7816089BF80B5826080BD8BB7806229
S11312E08BBFE9ECF0E080818D60808384E89EE12F
S11312F09093C5008093C400899A8AB38F688ABB8F
S1131300BA98E2E6F0E0808184608083B3D6789472
S1131310C2D6882309F40BC104DE60911A017091CE
S11313201B0180E090E0F9D16091180170911901DE
S113133082E090E0F2D1609116017091170188E18A
S113134090E0EBD1609114017091150184E090E07C
S1131350E4D1609112017091130186E090E0DDD137
S113136060911001709111018AE190E0D6D16091F1
S11313700E0170910F0188E090E0CFD160910C01D3
S113138070910D018AE090E0C8D160910A017091DA
S11313900B018CE090E0C1D16091080170910901CA
S11313A08EE090E0BAD1609106017091070180E16E
S11313B090E0B3D1609104017091050182E190E065
S11313C0ACD1609102017091030184E190E0A5D158
S11313D0609100017091010186E190E09ED16091DD
S11313E01C018CE190E08BD180E090E083D190935C
S11313F01B0180931A0182E090E07CD19093190143
S11314008093180188E190E075D19093170180933F
S1131410160184E090E06ED190931501809314013D
S113142086E090E067D190931301809312018AE1E2
S113143090E060D1909311018093100188E090E0D6
S113144059D190930F0180930E018AE090E052D11C
S113145090930D0180930C018CE090E04BD190931C
S11314600B0180930A018EE090E044D1909309012E
S11314708093080180E190E03DD19093070180932F
S1131480060182E190E036D1909305018093040136
S113149084E190E02FD1909303018093020186E1CF
S11314A090E028D190930101809300018CE190E0B9
S11314B019D180931C013BC081E0CCDC49D98A83DB
S11314C09ED989838A81082E000C990B9093500130
S11314D080934F018981082E000C990B90934E0143
S11314E080934D01D89A69818A81E0D969818A8182
S11314F047DB6091210170E080E090E049D8609181
S11315003C0170E080E090E07BD86091200170E0C5
S113151080E090E0ADD860911F0170E080E090E041
S1131520DFD88FE097E20197F1F700C000008091C7
S113153045018111C1CF8FE08DDCF9CFAA1BBB1B04
S113154051E107C0AA1FBB1FA617B70710F0A61BBF
S1131550B70B881F991F5A95A9F780959095BC01E0
S1131560CD010895052E97FB16F400940FD057FD76
S113157005D068D007FC02D046F408C050954095C9
S1131580309521953F4F4F4F5F4F0895909580952B
S1131590709561957F4F8F4F9F4F08956894001306
S11315A0E894A0E0B0E0E6EDFAE01DC0EFEFE7F963
S11315B059016A015E23550FEE08FE2C87019B0139
S11315C0AC019E23990F660B762FCB015DD0CDB76E
S11315D0DEB7EAE024C02F923F924F925F926F925F
S11315E07F928F929F92AF92BF92CF92DF92EF92AF
S11315F0FF920F931F93CF93DF93CDB7DEB7CA1B30
S1131600DB0B0FB6F894DEBF0FBECDBF09942A885A
S1131610398848885F846E847D848C849B84AA8402
S1131620B984C884DF80EE80FD800C811B81AA818F
S1131630B981CE0FD11D0FB6F894DEBF0FBECDBF5A
S1131640ED010895A1E21A2EAA1BBB1BFD010DC0DA
S1131650AA1FBB1FEE1FFF1FA217B307E407F5075E
S113166020F0A21BB30BE40BF50B661F771F881F3A
S1131670991F1A9469F760957095809590959B01D0
S1131680AC01BD01CF010895DF93CF939F92A0E4F5
S11316909A2E0024D001E001F00116950795F794E5
S11316A0E794D794C794B794A79448F41068A20F0A
S11316B0B31FC41FD51FE61FF71F081E191E220FD4
S11316C0331F441F551F661F771F881F991F9A9445
S11316D021F79D01AE01BF01C00111249F90CF915C
S11316E0DF910895E199FECF9FBB8EBBE09A9927C5
S11316F08DB30895A8E1B0E042E050E013C0262F76
S1131700E199FECF1CBA9FBB8EBB2DBB0FB6F894DC
S1131710E29AE19A0FBE01960895F1DF272FF0CFE8
S1131720DC01CB01FC01E199FECF06C0FFBBEEBB9F
S1131730E09A31960DB20D9241505040B8F7089599
S1071740F894FFCF47
S1131744D007E803D007E803D007E803D007E80389
S1131754DC05D007E803DC05D007E8030301017FB7
S11317647F7FDF05DE05DD05DC05DF05DE05DD0540
S1091774DC050101010186
S9030000FC
